:1000000012C02CC02BC02AC029C028C027C026C0BF
:1000100025C024C023C022C021C020C01FC01EC0D4
:100020001DC01CC01BC011241FBECFE5D4E0DEBF25
:10003000CDBF10E0A0E6B0E0EEEDF1E002C005902B
:100040000D92A036B107D9F710E0A0E6B0E001C0EC
:100050001D92A037B107E1F758D0C0C0D1CFAC0195
:10006000892B59F020E030E08AEF90E00197F1F71A
:100070002F5F3F4F24173507B9F70895BB9ABC98F7
:10008000BD9A8A98BA9AA19A8B9A0895C29AC39AED
:10009000C59880B386B3A99A0895C598C29840E0E0
:1000A00020E030E0992314F4C39A01C0C398C59AA4
:1000B000220F331FB4992160C5984F5F403119F06A
:1000C000880F991FEFCFC598C29AC90108958299E8
:1000D000FECF90E080509844E0DF08958299FECFF3
:1000E00080E090E0DADF80E090EBD7DF90E00895E9
:1000F00010BC8CE089B988E18AB986E880BD599A3C
:1001000008955D9BFECF8CB908956F927F929F9268
:10011000AF92BF92CF92DF92EF92FF920F931F9315
:10012000CF93DF93ABDFB2DFE3DF939A88EE93E008
:1001300096DF939887EE90E8B0DF89ED92E8ADDF27
:1001400080E496EAAADF83E296ECA7DF8AEC90E9E6
:10015000A4DF8CEA92ECA1DF81E89AEC9EDF84EDCB
:100160009EEC9BDF8BE694EC98DF87E59CEC95DFBB
:1001700099240F2EF0E6AF2EF0E0BF2EF02D3501C2
:10018000CC24DD246894C4F8CA0CDB1C83E89AEC08
:1001900084DF8501E301FF24A1DF8993F80ECC15EC
:1001A000DD05D1F79BDFE82E99DF80E09AEC75DF63
:1001B000F80181918F01A5DF82E090E050DFC01748
:1001C000D107B1F7FE1411F4909402C08CE099DFCE
:0E01D000992011F0939ADACF9398D8CFFFCFF1
:00000001FF
